:10000000F331F2BD3E00ED39393E10ED39383E8A0C
:10001000ED393A1875436972637569742043656CEC
:100020006C617220486F6D6520436F6E74726F6CE7
:100030002053797374656D2049492D2D5375706572
:10004000727669736F727920436F6E74726F6C6C25
:1000500065722D2D56657273696F6E20312E3230A8
:100060002D2D436F70797269676874202863292089
:10007000313939322C2043697263756974204365C4
:100080006C6C61722C20496E632ECD1A1BCD2E1C18
:10009000CD0A1CCD1E1CCDED1BCD991CCDB21CCDA7
:1000A000941BCDC21CCDBD1BCD7E1B217FBD8628E0
:1000B00003CD631B3EFF3210BDCD621CCD521D210E
:1000C000B3011132BE0100203E01CDA91E21370E21
:1000D0001172BE0100203E02CDA91E217A0F11B27D
:1000E000BE0100203E03CDA91E21311011F2BE0138
:1000F00000203E04CDA91E21E8111132BF010020CD
:100100003E05CDA91E21A7141172BF0100203E0695
:10011000CDA91E21121611B2BF0100203E07CDA9A4
:100120001E21DB1611F2BF0100203E08CDA91E21C1
:10013000A1171132C00100203E09CDA91E2154187B
:100140001172C00100203E0ACDA91E21141911B25E
:10015000C00100203E0BCDA91E1101003E01CDC300
:100160001E1164003E02CDC31E110A003E03CDC322
:100170001E110A003E04CDC31E1132003E05CDC340
:100180001E1101003E06CDC31E1130003E07CDC337
:100190001E1131003E08CDC31E1133003E09CDC3F0
:1001A0001E1134003E0ACDC31E1135003E0BCDC3D7
:1001B0001E18FE3132BECD4702CD9002DD21F2C0C5
:1001C000DD7E00FEFFCA3F02DD7E00FEF12004DD81
:1001D000231865FEF02026DD23CD6B08DD23205893
:1001E000DD7E00DD23FEF82004DD2318F3FEF92078
:1001F00006DD23DD2318E9FEF120E5183BCD6B0871
:100200002814DD7E00F53EFFDD7700DD23F1B72009
:100210000CCDA10218223E00DD7700DD23DD7E003B
:10022000DD23FEF82004DD2318F3FEF92006DD238C
:10023000DD2318E9FEFE20E5DD7E00FEFF20893E7D
:10024000003210BDC3B601DD2100A2FD2100A321B3
:1002500000A41100A50600F3DD7E00FD77007E36C8
:100260000012FBDD23FD23231310ECDD2100A6FD8E
:100270002100A72100A81100A90600F3DD7E00FDE2
:1002800077007E360012FBDD23FD23231310ECC91B
:10029000C50102C9ED78EE80ED7901FFDFED78C18F
:1002A000C9C5D5E5DD7E00FEFECA1207FE80DA2252
:1002B00003CA3C03FE81CA4003FE90CAAF03FE910D
:1002C000CAB303FEA0CA5E03FEA1CA6203FEA2CAAD
:1002D0007503FEA3CA8D03FEA4CA9E03FE94CAF64C
:1002E00003FE95CAFA03FEB0CAFB04FEB1CA52056A
:1002F000FEB2CAF105FEB3CAAA05FE98CA4706FEB9
:1003000088CAC906DD23DD7E00FEF82004DD23183F
:10031000F3FEF92006DD23DD2318E9FEFE20E5C308
:100320001207DD4600DD4E01DD5602DD5E03CD2EF7
:1003300007DD23DD23DD23DD23C3A4023EFF1802F6
:100340003E002100ABDD5E01160019772140ABCBEA
:1003500023193E00772377DD23DD23C3A4023EFF6C
:1003600018023E0021C0ABDD5E0116001977DD23C7
:10037000DD23C3A402DD7E0321C0ABDD5E011600D8
:100380001977DD23DD23DD23DD23C3A40221C0ABE8
:10039000DD5E0116001934DD23DD23C3A40221C074
:1003A000ABDD5E0116001935DD23DD23C3A4021683
:1003B000FF18021600211807DD7E01CB3FCB3FCB93
:1003C0003FCB2706004F094E2346C5DD7E01E607D9
:1003D0003C47AF371710FDC1ED58CB422803B31887
:1003E000022FA3ED792100AADD4E0106000972DD7E
:1003F00023DD23C3A402160118021600D53A4BBD13
:10040000B720FADD7E01FE403867FE60DAC80411CD
:10041000C0AD21CF04011800EDB0DD7E01D6600E25
:1004200000D61838030C18F9C6184779C63032C9F7
:10043000AD780F0F0FE603C63032D0AD78E607C6B1
:100440003032D2ADD17AC63032D4AD2100A6FD21F2
:1004500000A8DD4E01060009FD097E72BA2804FDE0
:100460003600FF21C1ADCDC51A3A7BBDB72859185A
:100470004D11C0AD21E704011400EDB0DD7E010F88
:100480000F0FE607C63032C8ADDD7E01E607C63085
:1004900032CEADD17AC63032D0AD2100A6FD2100DA
:1004A000A8DD4E01060009FD097E72BA2804FD365A
:1004B00000FF21C1ADCDC51A3A7ABDB7280A3E006A
:1004C000324CBD3EFF324BBDDD23DD23C3A4020D04
:1004D000233030204144494F3020534450302E3097
:1004E0002E303D300D0A000D2330302044494F306E
:1004F000205344502E303D300D0A003A4BBDB720FA
:10050000FA11C0AD214405010D00EDB021CDADDDE6
:1005100023DD7E00DD23C63032C9ADDD7E00DD2364
:100520007723FE0D20F5360A23360021C1ADCDC557
:100530001A3A79BDB7280A3E00324CBD3EFF324B15
:10054000BDC3A4020D233030205445524D302053FA
:100550003D003A4BBDB720FA11C0AD219B05010EFD
:1005600000EDB021CEADDD23DD7E00DD23C63032CF
:10057000C8ADDD7E00DD237723FE0D20F5360A238E
:10058000360021C1ADCDC51A3A7ABDB7280A3E0062
:10059000324CBD3EFF324BBDC3A4020D2330302090
:1005A00044494F30205444503D003A4BBDB720FAE7
:1005B00011C0AD21E705010900EDB021C9ADDD2372
:1005C000DD7E00DD23C63032C5ADDD7E00DD237764
:1005D00023FE0D20F5360A2336003E00324CBD3E88
:1005E000FF324BBDC3A4020D212054563020533D91
:1005F000003A4BBDB720FA11C0AD213506011200FB
:10060000EDB021CBADDD23DD7E00DD23C63032C76A
:10061000AD0604DD7E00DD23772310F721C1ADCDCB
:10062000C51A3A78BDB7280A3E00324CBD3EFF32AB
:100630004BBDC3A4020D2330302049523020534D0E
:10064000303030310D0A003A4BBDB720FA11C0AD41
:1006500021B206011700EDB0DD7E010F0FE607C6DF
:100660003032C9ADDD7E01E603C63032D0ADDD7E6D
:1006700003470F0F0F0FE60FC630FE3A3802C607CA
:1006800032D2AD78E60FC630FE3A3802C60732D312
:10069000AD21C1ADCDC51A3A7BBDB7280A3E0032A7
:1006A0004CBD3EFF324BBDDD23DD23DD23DD23C307
:1006B000A4020D233030204144494F302053414F94
:1006C000302E303D30300D0A003A4BBDB720FA11C4
:1006D000C0AD210307010F00EDB0DD7E01CD55084F
:1006E00021CAAD70237121C1ADCDC51A3A77BDB70E
:1006F000280A3E00324CBD3EFF324BBDDD23DD23D8
:10070000C3A4020D23303020583130205230300D38
:100710000A00DD23E1D1C1C9028010A010A011A000
:1007200012A000C901C902C900E801E802E8DDE53C
:100730007AFE03200CCDFB07C2D8077ACD15081826
:1007400024FE052005CD1508181BFE062005CD1535
:10075000081812FE0420047ACD3408FE012804FE95
:100760000220020E013A4BBDB720FAC5D511C0AD2B
:1007700021E707011400EDB0D1C1DD21C0ADDD706E
:100780000A79CD5508DD700BDD710C21DB07060001
:100790004A0DCB210946234EDD700DDD710E7BCD58
:1007A00055087AFE062815FE0528113E0DDD770F47
:1007B0003E0ADD77103E00DD77111806DD700FDD93
:1007C000711021C1ADCDC51A3A77BDB7280A3E00D8
:1007D000324CBD3EFF324BBDDDE1C94146414E4F7B
:1007E0004E4F46444D42520D233030205831302078
:1007F000534130314F4E30300D0A00D5E578D641A7
:1008000017171717E6F0813D5F16002100A1197E2A
:10081000E67FE1D1C9F5D5E578D64117171717E678
:10082000F0813D5F16002100A1193EFF773245BDE2
:10083000E1D1F1C9F5D5E578D64117171717E6F0DC
:10084000813D5F16002100A1193E80773EFF3245B1
:10085000BDE1D1F1C9F5010000D60A38030418F949
:10086000C60AC6304F78C63047F1C9C5D5FD21024A
:10087000A0CDA30847DD7E00DD23FEFD2820FE2954
:10088000281C57CDA3084F7AFE2A2808FE2B2809DA
:100890000600180A78A14718DC78B14718D778B74E
:1008A000D1C1C9C5D5E50600DD7E00DD23FE7E2071
:1008B0000406FF18F3FE28CA8609FED8CA900CFE6B
:1008C000B0CADA0CFEB1CAEB0CFEB2CAFC0CFE8058
:1008D000CA8C09FE81CACA09FE82CA080AFE83CAF6
:1008E000460AFE84CA840AFE90CAC20AFE91CAED74
:1008F0000AFE92CA180BFE93CA440BFE94CA700BF0
:10090000FE98CA960CFE99CAA70CFEA0CA9B0BFEC5
:10091000A1CAAF0BFEA2CAC30BFEA3CAD70BFEA48B
:10092000CAEB0BFE88CAFF0BFE89CA1C0CFE8ACAE2
:10093000390CFE8BCA560CFE8CCA730CFED0CAC68C
:100940000DFED1CAE30DFEB8CAB80CFEB9CAC90C77
:10095000FEB4CA0D0DFEB5CA1E0DFEB6CA2F0DFEA1
:10096000C0CA400DFEC1CA540DFEC2CA680DFEC306
:10097000CA7C0DFEC4CA900DFEC8CAA40DFEC9CA29
:10098000B50DAFC3320ECD6B08C3320EDD7E00FD58
:10099000BE00C2160EDD7E01FDBE01C2160EDD7E5A
:1009A00002B7CA1A0EFE08200A3A12BDB7C21A0EC2
:1009B000C3160EFE09200A3A13BDB7C21A0EC3169B
:1009C0000EFDBE02C2160EC31A0EDD7E02B728202F
:1009D000FE0820093A12BDB72016C3160EFE0920E4
:1009E000093A13BDB72009C3160EFDBE02C2160E8A
:1009F000FD7E01DDBE01DA160EC21A0EDD7E00FD9F
:100A0000BE00D2160EC31A0EDD7E02B72820FE08E5
:100A100020093A12BDB72016C3160EFE0920093A66
:100A200013BDB72009C3160EFDBE02C2160EDD7E31
:100A300001FDBE01DA160EC21A0EFD7E00DDBE00FB
:100A4000D2160EC31A0EDD7E02B72820FE0820093A
:100A50003A12BDB72016C3160EFE0920093A13BD7F
:100A6000B72009C3160EFDBE02C2160EFD7E01DDC3
:100A7000BE01DA160EC21A0EFD7E00DDBE00DA16C9
:100A80000EC31A0EDD7E02B72820FE0820093A1296
:100A9000BDB72016C3160EFE0920093A13BDB720B4
:100AA00009C3160EFDBE02C2160EDD7E01FDBE019B
:100AB000DA160EC21A0EDD7E00FDBE00DA160EC377
:100AC0001A0E2100ABDD5E001600197EB7CA240E97
:100AD0002140ABDD5E00CB231600195E2356DD6E90
:100AE00002DD6603AFED52CA280EC3240E2100AB0F
:100AF000DD5E001600197EB7CA240E2140ABDD5E14
:100B000000CB231600195E2356DD6E02DD6603AFAF
:100B1000ED52DA280EC3240E2100ABDD5E00160074
:100B2000197EB7CA240E2140ABDD5E00CB23160030
:100B3000195E2356DD6E02DD6603EBAFED52DA2857
:100B40000EC3240E2100ABDD5E001600197EB7CA6D
:100B5000240E2140ABDD5E00CB231600195E235628
:100B6000DD6E02DD6603EBAFED52D2280EC3240E1C
:100B70002100ABDD5E001600197EB7CA240E2140AD
:100B8000ABDD5E00CB231600195E2356DD6E02DD61
:100B90006603AFED52D2280EC3240E21E0ABDD5E1A
:100BA000001600195EDD7E0293CA1A0EC3160E21CE
:100BB000E0ABDD5E001600195EDD7E0293DA1A0EF0
:100BC000C3160E21E0ABDD5E001600197EDD5E026D
:100BD00093DA1A0EC3160E21E0ABDD5E0016001983
:100BE0007EDD5E0293D21A0EC3160E21E0ABDD5EEF
:100BF000001600195EDD7E0293D21A0EC3160E2176
:100C000060ACDD5E011600195E3600CB7BCA160EA5
:100C1000CBBBDD7E0293CA1A0EC3160E2160ACDD7B
:100C20005E011600195E3600CB7BCA160ECBBBDD0B
:100C30007E0293DA1A0EC3160E2160ACDD5E011639
:100C400000197E3600CB7FCA160ECBBFDD5E029345
:100C5000DA1A0EC3160E2160ACDD5E011600197E95
:100C60003600CB7FCA160ECBBFDD5E0293D21A0EC2
:100C7000C3160E2160ACDD5E011600195E3600CB96
:100C80007BCA160ECBBBDD7E0293D21A0EC3160EA4
:100C90003A10BDC3320E2100ABDD5E001600197E96
:100CA000B7CA000EC3040E2100ABDD5E00160019AA
:100CB0007EB7C2000EC3040E2100AADD5E0016003E
:100CC000197EB7CA000EC3040E2100AADD5E00160D
:100CD00000197EB7C2000EC3040E2100A3DD5E0022
:100CE0001600197EB7CA000EC3040E2100A3DD5EF4
:100CF000001600197EB7C2000EC3040E2100A5DD48
:100D00005E001600197EB7CA000EC3040E2100A7AC
:100D1000DD5E001600197EB7CA000EC3040E210066
:100D2000A7DD5E001600197EB7C2000EC3040E21B7
:100D300000A9DD5E001600197EB7CA000EC3040EBE
:100D400021C0ABDD5E001600195EDD7E0293CA1A7B
:100D50000EC3160E21C0ABDD5E001600195EDD7EEF
:100D60000293DA1A0EC3160E21C0ABDD5E00160028
:100D7000197EDD5E0293DA1A0EC3160E21C0ABDDBA
:100D80005E001600197EDD5E0293D21A0EC3160EA7
:100D900021C0ABDD5E001600195EDD7E0293D21A23
:100DA0000EC3160E21C0ABDD5E001600197EB7CA59
:100DB000000EC3040E21C0ABDD5E001600197EB725
:100DC000C2000EC3040EDD7E00D64117171717E6CA
:100DD000F0DD86013D5F16002100A1197ECB47287A
:100DE00029182BDD7E00D64117171717E6F0DD8690
:100DF000013D5F16002100A1197ECB47200C180E83
:100E00003E0018023EFFDD2318283E0018023EFF78
:100E1000DD23DD23181C3E0018023EFFDD23DD2309
:100E2000DD23180E3E0018023EFFDD23DD23DD2307
:100E3000DD23A8E1D1C1C9F33172BE3A01A05F3A06
:100E400002A057D506083A80BD10FB21E0110E081C
:100E500006087E3280BD0F10FA230D20F306083AF3
:100E600080BD1FCB1910F879D947D906083A80BD43
:100E70001FCB1910F879D94FD906083A80BD1FCB7E
:100E80001910F879D957D906083A80BD1FCB191027
:100E9000F879D95FD906083A80BD1FCB1910F879C7
:100EA000E60FD967D906083A80BD1FCB1910F8792B
:100EB000D96FD906083A80BD1FCB1910F851060822
:100EC0003A80BD1FCB1910F859DD2100A0DD720654
:100ED000DD7307D9DD7000DD7101DD7202DD7303A2
:100EE000DD7404DD7505D9FBD13A02A0BAC4540FF4
:100EF0003A01A0BB2835CD2E0F3A04A0FE012804EC
:100F0000FE07200C3EFF3213BD3E003212BD180A10
:100F10003EFF3212BD3E003213BD3EFF3241BD32B4
:100F200042BD3243BD3244BD3246BDC3DD1EDD216C
:100F300040AB2100AB06207EB72811DD5E00DD56F8
:100F400001137AB32806DD7300DD720123DD23DD92
:100F50002310E4C9DD2180AB2120AB06207EB72819
:100F600011DD5E00DD5601137AB32806DD7300DD66
:100F7000720123DD23DD2310E4C931B2BE2100A2BA
:100F8000FD2100A4DD210D10DD4E00DD460178B10C
:100F900028231E08ED503EFFCB3A38023E00C546DE
:100FA000B82804FD3600FFC17723FD231D20E7DDAF
:100FB00023DD2318D33A7CBDB7284BFE033028012C
:100FC00000903A11BD814FED5821E0AB3A11BD06BA
:100FD000004F09733CFE0838023E003211BD01008B
:100FE00090814FED79181F0100903A11BD814FEDAE
:100FF0005821E8AB3A11BD06004F09733CFE083892
:10100000023E003211BD210FBD34C3DD1E00800140
:101010008000A001A002A000C801C802C800EB0126
:10102000EB02EB00EA01EA02EA00E901E902E90069
:101030000031F2BECD9814CA1311CD9E14FE21C208
:101040001311CD2A113E5ECD8B14CD9E14FE3D288A
:1010500019FE23C210112108A0CD9E1477FEFF288F
:10106000032318F5CD4011C310113E01CD0A1FCD49
:101070009E14327CBD2177BD0605CD9E14772310CA
:10108000F9CD9E146FCD9E1467227DBD1E00060013
:1010900021F2C0CD9E147780477BB728031D181519
:1010A0007EFEF820041E01180CFEF920041E021812
:1010B00004FEFF28032318DBCD9E14327FBD802859
:1010C00005CD631B18053E5ECD8B14CD991CCD62FA
:1010D0001C3EFF3210BD1101003E01CDC31ECD35B7
:1010E000113A7BBDB7282C470E003A57BDB720FAFE
:1010F000C521161111E0AE011400EDB0C179C63062
:1011000032E7AE3E003258BD3EFF3257BD0C10DA1A
:10111000CD3511C3DD1E0D21204144494F302044FF
:1011200050302E333D39320D0A00F3ED3810CB87A5
:10113000ED3910FBC9F3ED3810CBC7ED3910FBC901
:10114000F3C5D5E5D9C5D5E5DD2108A0DD4600DD2F
:101150004E01DD5602DD5E03DD6604DD6E05D9DD80
:101160005606DD5E0706083A80BD10FB21E0110E31
:101170000806087E3280BD0F10FA230D20F3D978BF
:10118000D906083280BD0F10FAD979D90608328005
:10119000BD0F10FAD97AD906083280BD0F10FAD9DE
:1011A0007BD906083280BD0F10FAD97CD9CBAFCBE2
:1011B000E706083280BD0F10FAD97DD906083280C3
:1011C000BD0F10FA7A06083280BD0F10FA7B0608B0
:1011D0003280BD0F10FAD9E1D1C1D9E1D1C1FBC92B
:1011E000C53AA35CC53AA35C3132BF3A41BDB7C42E
:1011F00036123E003241BD3A42BDB7C44E123E00E7
:101200003242BD3A43BDB7C4DF123E003243BD3A5D
:1012100044BDB7C465133E003244BD3A45BDB7C4B2
:1012200095133E003245BD3A46BDB7C4DA133E00C1
:101230003246BDC3DD1EF5C5E53E23CD8B1421002E
:10124000A006087ECD8B142310F9E1C1F1C9C5E5D4
:101250003A7CBDB7CADC12FE0330323E3CCD8B1463
:101260003E30CD8B142100A20602CD4F133E00CD9F
:101270008B143A7CBDFE0220633E3CCD8B143E3184
:10128000CD8B142110A20603CD4F13184F3E3CCD39
:101290008B143E32CD8B142128A20603CD4F133A76
:1012A0007CBDFE0420363E3CCD8B143E33CD8B14EA
:1012B0002140A20603CD4F133E3CCD8B143E34CDCE
:1012C0008B142158A20603CD4F133E3CCD8B143E08
:1012D00035CD8B142170A20603CD4F13E1C1C9C5D2
:1012E000E53A7CBDB7CA4C13FE0330353E7DCD8B4D
:1012F000143E36CD8B142100AA0601CD4F133E00BB
:10130000CD8B14CD8B143A7CBDFE02203F3E7DCDAB
:101310008B143E37CD8B142110AA0603CD4F131822
:101320002B3E7DCD8B143E38CD8B142128AA06038D
:10133000CD4F133A7CBDFE0420123E7DCD8B143E72
:1013400039CD8B142140AA0603CD4F13E1C1C9F555
:10135000C50E0006087E1FCB192310F979CD8B141A
:10136000C110EDF1C93A7CBDB72829FE03300F3E0C
:101370007ECD8B143E00CD8B1421E0AB180D3E7E4C
:10138000CD8B143E08CD8B1421E8AB06087ECD8BA7
:10139000142310F9C92A7DBD06100E41CB3CCB1D8C
:1013A00030093E3ECD8B1479CDAF130C10EEC9C57C
:1013B000D5E5CD8B14D6414F0610ED4C2100A10987
:1013C00011000006107E1FCB1ACB1B2310F77BCD1C
:1013D0008B147ACD8B14E1D1C1C9DD2177BD2114E5
:1013E000BD06050E08DD56001E007AB7281E3E2AEF
:1013F000CD8B143E0690CB27CB27CB27CB27B3CD65
:101400008B147ECD8B14231C0D1520DE79B7280498
:10141000230D18F8DD2310CBC9F51F1F1F1FE60F82
:10142000FE0A3802C607C630CD8B14F1F5E60FFE72
:101430000A3802C607C630CD8B14F1C9F5C5D501EF
:1014400000001600D66438030418F9C664D60A38BA
:10145000030C18F9C60A5778C630CD8B1479C630FC
:10146000CD8B147AC630CD8B14D1C1F1C9F53E0DA8
:10147000CD8B143E0ACD8B14F1C9E3F5CD8214F166
:10148000E3C97E23B7C8CD8B1418F7F5ED3805CB2B
:101490004F28F9F1ED3907C9ED3805E680C9CD9837
:1014A0001428FBED3809C93172BFDD2147BD21E0A9
:1014B000B1220ABD2160AD2208BD060C3A4BBDB772
:1014C0002838DDE5DD214BBD2A0ABDE521A0B22289
:1014D0000ABD2A08BDE521C0AD2208BDF3CD3315F4
:1014E000FBDD7E01B72803CD8415DD360000E12247
:1014F00008BDE1220ABDDDE118C2DD7E00B7281279
:10150000F3CD3315FBDD7E01B72803CD8415DD3621
:101510000000DD23DD23DD23DD232A0ABD11C00009
:1015200019220ABD2A08BD116000192208BD108CBD
:10153000C3AA14C5E52A08BDCD4D1506607EB7289F
:1015400006CD5C152310F6CD6915E1C1C9C5ED00C6
:1015500000CBA0ED0100063210FEC1C9F5ED380444
:10156000CB4F28F9F1ED3906C9C5ED0004CB482869
:10157000F90E05060010FE0D20FBED0000CBE0ED9E
:101580000100C1C9C5D5E53E00320FBD2A0ABD2202
:101590000CBD3E00320EBD2A00BDEB2A02BD7DBB54
:1015A000282E7E472C2202BDFE0A2837FE0D283346
:1015B0003A0EBDFEC030082A0CBD78FE2420082A51
:1015C0000ABD3E00320EBD7023220CBD210EBD347B
:1015D0003A0FBDFE0538C03E00DD77023EFFDD77E5
:1015E0000318263A0EBDB728AE2A0CBD36002322BA
:1015F0000CBD210EBD340E28060010FE0D20FB3E52
:1016000000DD77033EFFDD77023E00DD7701E1D1AB
:10161000C1C931B2BF3A77BDB7CAB2161100B02105
:10162000BD16010E00EDB02101B0CDC51A3EFF324E
:1016300064BD3263BD3A65BDB7200D3A66BDB728BB
:10164000F43E003214BD186A2120B7CDF11A2807E4
:101650003E023214BD185B3E013214BD2128B7DDB5
:101660002100A106107ECDCB160707070757237E62
:10167000CDCB16B257237ECDCB16070707075F23C6
:101680007ECDCB16B35F23C506100E7FCB3ACB1BA6
:1016900038020E00DD7E00E67FB92807DD7E00CB34
:1016A0007F2003DD7100DD2310E0C110B83EFF3262
:1016B00045BD3E003265BD3266BDC3DD1E0D233023
:1016C00030205831302051530D0A00D630FE0AD850
:1016D000D607C9C630FE3AD8C607C931F2BF3A7933
:1016E000BDB7CA8717473A3EBDB838053E00323EFF
:1016F000BD1160B0219217010F00EDB03A3EBDC69A
:10170000303269B02161B0CDC51A3EFF3268BD32BA
:1017100067BD3A69BDB720142124BD3A3EBD5F16AE
:1017200000193A6ABDB728EA36001857E521E0B734
:10173000CDF11AE128043602184D360121EAB77EB0
:10174000CDCB16070707074F237ECDCB16B14F3AF7
:101750003EBDE60707072140A6FD2140A85F160011
:1017600019FD190604CB39CB39CB39CB393E00CB27
:101770003930023E015677BA2804FD3600FF23FDBA
:101780002310EA213EBD343E003269BD326ABDC33A
:10179000DD1E0D233030205445524D3020510D0AAE
:1017A000003132C03A78BDB7CA3718473A3DBDB8A4
:1017B00038053E00323DBD11C0B021421801120073
:1017C000EDB03A3DBDC63032C7B021C1B0CDC51A6B
:1017D0003EFF326CBD326BBD3A6DBDB72014211C8B
:1017E000BD3A3DBD5F1600193A6EBDB728EA360016
:1017F0001841E521A0B8CDF11AE1280436021837C6
:1018000036013A3DBDCBFF5F21B1B8DD2160AC06AA
:10181000207ECDCB16070707074F237ECDCB16B111
:101820004F23C50608CB393003DD7300DD2310F5E7
:10183000C110DE213DBD343E00326DBD326EBDC3F0
:10184000DD1E0D233030204952302051302D3235ED
:10185000350D0A003172C03A7ABDB7CAF918473A55
:101860003FBDB838053E00323FBD1120B1210419FB
:10187000011000EDB03A3FBDC6303228B12121B190
:10188000CDC51A3EFF3270BD326FBD3A71BDB72073
:1018900014212CBD3A3FBD5F1600193A72BDB7281E
:1018A000EA36001850E52160B9CDF11AE128043676
:1018B0000218463601216CB97ECDCB160707070703
:1018C0004F237ECDCB16B14F3A3FBDE60707070742
:1018D0002100A6FD2100A85F160019FD1906083E8B
:1018E00000CB3930023E015677BA2804FD3600FF9E
:1018F00023FD2310EA213FBD343E003271BD327218
:10190000BDC3DD1E0D2330302044494F30205144EB
:10191000500D0A0031B2C03A7BBDB7CA201A473A0F
:1019200040BDB838053E003240BD1180B1212B1AB0
:10193000012000EDB03A40BDC6303289B12181B1FD
:10194000CDC51A3EFF3274BD3273BD3A75BDB720A6
:10195000152134BD3A40BD5F1600193A76BDB7284F
:10196000EA3600C31C1AE52120BACDF11AE1280499
:101970003602183A36012130BACD891A2160A6FD07
:101980002160A8CD9D1A2139BACD891A2168A6FDFA
:101990002168A8CD9D1A2142BACD891A2170A6FDD1
:1019A0002170A8CD9D1A3E003275BD3276BD1180E2
:1019B000B1214B1A013E00EDB03A40BDC63032892C
:1019C000B12181B1CDC51A3EFF3274BD3273BD3A2B
:1019D00075BDB720142134BD3A40BD5F1600193AD9
:1019E00076BDB728EA36001833E52120BACDF11AC2
:1019F000E128043602182936013A40BDE6070707F8
:101A00000721F0AB5F1600191130BA0608EBCD893B
:101A10001AC501090009C1EB772310F12140BD343B
:101A20003E003275BD3276BDC3DD1E0D2330302041
:101A30004144494F3020514450302E302C445030D6
:101A40002E312C4450302E320D0A000D2330302020
:101A50004144494F3020514149302E302C414930CA
:101A60002E312C4149302E322C4149302E332C411D
:101A700049302E342C4149302E352C4149302E36F8
:101A80002C4149302E370D0A00C5E57ECDCB160717
:101A90000707074F237ECDCB16B1E1C1C94F3A40AE
:101AA000BDE6070707075F160019FD1906083E0087
:101AB000CB3930023E015677BA2804FD3600FF23A9
:101AC000FD2310EAC9C5E50E007E23FE0D2808FEA1
:101AD0000A2804814F18F2792F3C4FE1231F1F1F62
:101AE0001FE60FCDD316772379E60FCDD31677C136
:101AF000C9C5237ECDCB1617171717E6F047237EEF
:101B0000CDCB16B04736302B36302B0E007E23B7A8
:101B10002804814F18F77980C1C9C5D5E521A0BD3A
:101B2000ED29337CED470609112B1D732372231019
:101B3000FA3E00215D1B010006ED93ED3808ED38FB
:101B4000093E0DED3906ED39073E60ED39323E00B4
:101B5000ED3934ED3936ED3910E1D1C1C974742154
:101B6000210000F5C5E53E01327FBD3EFF32F2C0E7
:101B70002177BD060836002310FBE1C1F1C9C5E598
:101B800021F2C006007E80477EFEFF28032318F561
:101B900078E1C1C9C5E521F2C07E23FEF820032308
:101BA0001813FEF920042323180BFEFF280CFEFD5A
:101BB00020033600237CFEFF20DFE1C1C9D5E521EB
:101BC00000BB2200BD2202BD21EB1C22AEBDED38C0
:101BD00004CBDFED39042100BC2204BD2206BD2167
:101BE0000B1D22B0BDED3805CBDFE1D1C9C5E5DD68
:101BF000E52100A4DD2100A806003E0077DD770086
:101C000023DD2310F7DDE1E1C1C9C5E52100A10114
:101C1000771C3E0077230B78B120F7E1C1C9C5E5F9
:101C20002100A106003E00772310FCE1C1C9C5E5F3
:101C300021441C4E23462378B128067E23ED7918D3
:101C4000F2E1C1C903809203A09B13A08003C89B4B
:101C500003C98003EB9B03EA9B03E99B03E8800035
:101C60000000F53A7CBDB72826FE033022ED38107F
:101C7000E6D1ED39103E01ED3914ED39163E00ED97
:101C80003915ED3917ED3810F606ED39101808ED55
:101C90003810E6D1ED3910F1C9C5E52100AB3E00A1
:101CA0000640772310FC2140AB0680772310FCE12F
:101CB000C1C9C5E521C0AB3E000610772310FCE189
:101CC000C1C9C5D5E521DE1C1160AD010D00EDB027
:101CD0003E003248BD3EFF3247BDE1D1C1C90D21B2
:101CE00020583130205230300D0A00F5E5ED38042F
:101CF000CB7F280BED38082A00BD772C2200BDEDE4
:101D00003800CB9FED3900E1F1FBC9F5E5ED380571
:101D1000CB7F280BED38092A04BD772C2204BDEDBA
:101D20003801CB9FED3901E1F1FBC9F5C5D5E5CD12
:101D30007A140D0A4843533A20496E7465727275DD
:101D40007074204572726F72210D0A00E1D1C1F1E9
:021D5000FBC9CD
:101D52002120A0221EA0E5DDE10610110F00AF3602
:101D62001023771910F9DD360004DD360320DD7704
:101D720006DD7707DD7702ED3810F611ED39103EFA
:101D820000ED390CED390E3E12ED390DED390FED46
:101D92005767ED3833F6046F36A123361DFBC9E5CC
:101DA200D5C5F5DDE5FDE5ED3810ED380CDD2A1E73
:101DB200A0DD360002FD2120A0111000FD7E00FEF4
:101DC20010282AFD6E06FD66077DB428072BFD75D7
:101DD20006FD7407FD6E08FD66097DB428072BFD1C
:101DE2007508FD7409FD1918D3F3111000210000C4
:101DF20039DD750CDD740DDD19DD7E00FE10200766
:101E0200DD2120A0DD7E00E60B28ECDD7E06DDB6BE
:101E12000720E4DD7E00FE012008DD7E08DDB60934
:101E220020D5DDE5FDE106020E00FD7E00E60B2871
:101E320025FD7E06FDB607201DFD7E00FE01200861
:101E4200FD7E08FDB609200EFD7E03B9FA581E2854
:101E5200054FFDE5DDE1FD19FD7E00FE1020CBFD05
:101E62002120A010C5DD221EA0DD6E0CDD660DF95D
:101E7200DD7E02ED3939DD7E00DD360004FE08200C
:101E82000BDD6E0ADD660BCD9F1EFBE9FE0220080C
:101E9200FDE1DDE1F1C1D1E1CD9F1EFBC9F5C50137
:101EA20000C0ED78C1F1C9CD261FDD360020DD71FD
:101EB20002DD7003DD750ADD740BDD730CDD720D5E
:101EC200C9F3CD261FDD7304DD7205DD7306DD72F5
:101ED20007DD360100DD360008FBC9F3DD2A1EA04E
:101EE200DD360020DD7E04DD7706DD7E05DD770749
:101EF200DD7E01B7C2EB1DDD360008C3EB1DF3DD4D
:101F02002A1EA0DD7003FBC9F3CD261FDD360101B9
:101F1200FBC9F3DD2A1EA0DD360001DD7308DD7288
:101F220009C3EB1DD5DD2120A01110003DFA361F9B
:061F3200DD1918F8D1C909
:00000001FF
